:100000000C94F6020C942E030C942E030C942E03E5
:100010000C942E030C942E030C942E030C942E039C
:100020000C942E030C942E030C94901F0C946220BD
:100030000C94CF190C942E030C942E030C942E03C5
:100040000C942E030C942E030C942E030C942E036C
:100050000C942E030C94571A0C942E030C942E031C
:100060000C942E030C942E030C942E030C942E034C
:100070000C942E030C942E030C942E030C942E033C
:100080000C942E030C942E030C942E030C942E032C
:100090000C942E030C942E030C942E030C942E031C
:1000A0000C942E030C942E030C942E03C807C8073F
:1000B000F407F4075C088709870987097A08130998
:1000C00024092409CF20F620EE21F620EE2142213A
:1000D0006521EE21BC21CB216D6F6465206A7573AB
:1000E0007420737769746368656420746F20717716
:1000F0006572747920616E64207468697320697315
:100100002061206875676520737472696E670A00E4
:100110002B0014001A000800150017001C0018001E
:100120000C00120013002A0029000400160007002A
:1001300009000A000B000D000E000F003300340010
:10014000E1001D001B000600190005001100100051
:100150003600370038002800AB5DE000E200E30025
:1001600003512C002C0004515000510052004F004C
:100170002B0014001A00090013000A000D000F00E4
:1001800018001C0033002A00290004001500160086
:10019000170007000B00110008000C0012003400CB
:1001A000E1001D001B000600190005000E001000F4
:1001B0003600370038002800AB5DE000E200E300C5
:1001C00003512C002C0004515000510052004F00EC
:1001D0002B0034003600370013001C0009000A0011
:1001E000060015000F002A00290004001200080074
:1001F00018000C0007000B00170011001600380053
:10020000E100330014000D000E001B00050010007B
:100210001A0019001D002800AB5DE000E200E300B9
:1002200003512C002C0004515000510052004F008B
:1002300035021E021F022002210222022302240292
:100240002502260227022A004C003A003B003C000F
:100250003D003E003F002D022E022F0230023102EF
:1002600001004000410042004300440045003202CA
:1002700064024A004D00010001000100010001007C
:100280000100010001000100AB00AA00A900AE00BE
:1002900035001E001F002000210022002300240042
:1002A0002500260027002A004C003A003B003C00B5
:1002B0003D003E003F002D002E002F003000310099
:1002C000010040004100420043004400450032006C
:1002D00064004B004E00010001000100010001001C
:1002E0000100010001000100AB00AA00A900AE005E
:1002F0001E001E001E001E001E001E001E001E000E
:100300001E001E001E001E00000014001A0008003F
:10031000150017001C0018000C00120013002F001D
:10032000000004001600070009000A000B000D0081
:100330000E000F0033003400AC5D0000000006002A
:100340001900000000001100100000000000000073
:100350000100005C015CC35CC45CC65CC75CC85C3B
:10036000C95CCA5CCB5C4C0001000100295C1D5CCF
:100370001E5C135C0A5CA75DA85DA95DAA5D010017
:1003800001002B5C2A5C265C275C2C5C2D5C000049
:100390000000010001000100010001000100010056
:1003A0000100010001000100010001000100010045
:1003B00044454255473A2064697361626C65642E16
:1003C0000A0044454255473A20656E61626C656497
:1003D0002E0A000A0025303258006C65645F746193
:1003E000736B3A20004F6E6573686F743A206163D7
:1003F000746976653A2025640A000A002530313692
:1004000062003A200025303258000A722F632030F3
:100410003132333435363738394142434445460A60
:10042000000A002530325820006B6579626F6172D6
:10043000645F7265706F72743A200064656C5F6B04
:1004400065795F6269743A2063616E277420646520
:100450006C3A20253032580A006164645F6B65791C
:100460005F6269743A2063616E2774206164643A44
:1004700020253032580A005B735D005B575D005BDE
:10048000535D005B525D005B445D005B435D000EAD
:100490000350006C0061006E0063006B0000000AF6
:1004A000034F004C004B0042000000040309040904
:1004B000025B00030100A0FA09040000010301012E
:1004C00000092111010001224000070581030800F5
:1004D00001090401000103000000092111010001CC
:1004E000226D0007058203200001090402000203B7
:1004F00000000009211101000122220007058303E9
:100500002000010705030320000112010002000082
:100510000008A80301AE0300010200010631FF0933
:1005200074A1010975150026FF0095207508810248
:100530000976150026FF00952075089102C0050177
:100540000980A101850319012AB700150126B7000A
:10055000950175108100C0050C0901A101850419E0
:10056000012AA002150126A002950175108100C084
:1005700005010906A1018506050719E029E715000F
:1005800025019508750181020507190029EF15005D
:10059000250195F0750181020508190129059505C8
:1005A00075019102950175039101C005010906A12C
:1005B00001050719E029E715002501950875018156
:1005C000029501750881010507190029FF1500260C
:1005D000FF00950675088100050819012905950594
:1005E00075019102950175039101C00011241FBE90
:1005F000CFEFDAE0DEBFCDBF04B603FE18C08091B6
:10060000A3029091A402A091A502B091A602873006
:10061000904BA740B04B59F41092A3021092A40241
:100620001092A5021092A602E0E0F8E3099511E00D
:10063000A0E0B1E0E8E0F5E402C005900D92A23937
:10064000B107D9F722E0A2E9B1E001C01D92A33AB7
:10065000B207E1F70E94D2150C9482220C9400009C
:10066000FF93EF93E0919201F0919301309709F09D
:100670000995EF91FF910895FC018591803011F06B
:10068000EFDFFBCF0895FF27E0E230E247FF0CC029
:10069000419597FF09C0EDE2609570958095909522
:1006A000611D711D811D911D27FF02C0219530E341
:1006B00050E2AA27660F771F881F991FAA1FA41749
:1006C00010F0A41B63955A95A9F7AA3008F0A95F0A
:1006D000A05DAF93F395611571058105910541F713
:1006E000ED3211F4EF93F395F21718F43F93F3956D
:1006F000FBCF8F91B5DFFA95E1F70895E991F99174
:100700008591803021F0853219F0AADFF9CF089564
:1007100020E0E89455915532C1F3503311F46894B8
:1007200055915A3348F4505390F3220F022E220F62
:10073000220F200D250FF4CF0EF421958991999168
:10074000533619F3533729F1533559F1BC01882732
:100750009927E8945C3621F4899199916894559190
:10076000543639F446EF7EF077FF0DC08FEF9FEFE0
:100770000AC055374AE039F0583540E121F0523689
:1007800042E009F00895FF93EF937DDFEF91FF9131
:10079000B7CFFF93EF93FC0181918030B9F360DF15
:1007A000FBCFFF93EF9368DFF1CFDF93CF93CDB70C
:1007B000DEB72596A3DFCF91DF9108956E9A769AE2
:1007C0000C9483140F9306E024E043E00E94BE04DF
:1007D0000F910895CF93FB01893A2DE5920729F1F6
:1007E00040F4873A2DE5920771F0883A9D45A9F0CB
:1007F00056C08B3A2DE59207E9F030F18C3A9D45D1
:1008000009F445C04CC0C281CC2309F449C088ED2D
:1008100090E00E943C0380E005C0C281CC2309F433
:100820003FC081E00E94A40438C0C281CC23C1F142
:1008300082E0F8CFC28185EECC2319F00E945E06DB
:100840002CC00E9400072CC0C281CC2349F184E057
:100850000E94EC0A83E00E94EC0A86E00E94EC0A07
:1008600085E00E94CB0A0E946310811102C00E94A1
:1008700010110E947B109093810280688093800207
:1008800080918002909181020E948C1006C0C281EA
:10089000CC2331F085E00E94EC0AC0E001C0C1E049
:1008A0008C2FCF910895089581E008950C94EA0368
:1008B00008950C9458041F93CF93DF9300D000D079
:1008C0001F92CDB7DEB749835A836B833091950170
:1008D00089819A81311114C0662359F0222349F08D
:1008E0000E94C00B182F682F89819A810E94690B82
:1008F00003C00E94940B182F69817A81812F04C054
:100900000E94C00B69817A810F900F900F900F9019
:100910000F90DF91CF911F910C94FD12FC01262FB7
:10092000408151816281738184810C945B0481E0F8
:100930000895CF93DF93EC0160E00E948E04BE0126
:10094000DF91CF910C945904CF92DF92EF92FF92F6
:10095000C12CD12C7601C39404C0CC0CDD1CEE1C40
:10096000FF1C8A95D2F78C2D0E947610C701B60124
:10097000FF90EF90DF90CF900C946B0A8F929F9234
:10098000AF92BF92CF92DF92EF92FF920F931F939D
:100990006B017C0181E090E0A0E0B0E04C015D01E2
:1009A00004C0880C991CAA1CBB1C4A95D2F7AC0148
:1009B000BD0104C0440F551F661F771F2A95D2F74B
:1009C000482959296A297B2904C0880F991FAA1F21
:1009D000BB1F0A95D2F78A019B010C211D212E21F4
:1009E0003F21401751076207730739F4BC01CD015D
:1009F0006C297D298E299F290AC080959095A09504
:100A0000B095BC01CD016C217D218E219F211F91CC
:100A10000F91FF90EF90DF90CF90BF90AF909F909D
:100A20008F9008950C94DE030C94811408950E9415
:100A3000130A0E9416052FEF84E39CE021508040AA
:100A40009040E1F700C000000C947D1A0F931F93B3
:100A5000CF93DF938C0161E00E948E04EC01B8011A
:100A60000E945604882309F45BC0B801CE010E949D
:100A7000CB17882309F454C0B801CE010E94DF15BA
:100A8000882309F44DC0B801CE010E94271788239E
:100A900009F446C0F80182818823D9F1CF3D8CE565
:100AA000D80779F140F4C115FCE5DF0791F0C130BA
:100AB000DC4591F02EC0CC35EDE5DE0741F1CD35BA
:100AC000FDE5DF0709F1CB35DD4519F50E9457102B
:100AD00020C00E94170524C080914802C82FC095ED
:100AE000C170C0FB80F980934802CC2329F082ECCE
:100AF00093E00E943C0314C080EB93E00E943C030F
:100B000010C00E9410110CC00E944E1002C00E9422
:100B10005A10C801DF91CF911F910F910C9454048A
:100B2000C0E08C2FDF91CF911F910F9108950E940B
:100B3000B1190C94D5050E94D8050C94B71982956B
:100B4000982F937344E0949F900111248C7C869598
:100B50008695282B822F8575880F2A7A2695822BD9
:100B60000895CF93DF93D92F0E949F05C82F8D2F13
:100B70000E949F052C2F30E0322F2227A901482BFD
:100B8000CA01DF91CF91089508950C94C40581E0C6
:100B900008950C94C7050895CF93C82F0E94C505EA
:100BA0008C2F0E94C905CF91089580E00C94CC054C
:100BB0000E9427180C94CC05CF930E942718C82FA9
:100BC00080919401C81741F1C0939401809148022B
:100BD00082FF1EC080FF04C08AED93E00E943C03A8
:100BE0008091480280FF0CC01F92CF9385ED93E067
:100BF0009F938F930E94D5030F900F900F900F90AB
:100C00008091480280FF04C083ED93E00E943C0382
:100C10008C2FCF910C94CC05CF910895CF93DF9377
:100C2000CDB7DEB72B970FB6F894DEBF0FBECDBFA2
:100C30004F83588769877A878B8761110E94860F57
:100C40009E012F5F3F4F86E0F90111928A95E9F7E7
:100C500085E0FE013796D90101900D928A95E1F762
:100C600089819A814C815D81452B31F09F3F31F420
:100C700091E08F3F19F403C091E001C090E090FF34
:100C800009C049815A816B817C818D819E810E943E
:100C9000A70E05C0C9010E9497048111F2CF2B96BF
:100CA0000FB6F894DEBF0FBECDBFDF91CF91089590
:100CB000FC01808191810E94020C0895CF938823CA
:100CC00009F49CC0C82F8238C1F40E94271881FD06
:100CD00095C069E380910201909103010E946C1913
:100CE0000E94A80F2FEF81EE94E0215080409040A9
:100CF000E1F700C0000069E319C0833801F50E94E4
:100D0000271880FD7BC063E580910201909103016B
:100D10000E946C190E94A80F2FEF81EE94E02150E1
:100D200080409040E1F700C0000063E5809102013F
:100D3000909103010E947719CF910C94A80F8438E9
:100D4000C1F40E94271882FD59C067E48091020116
:100D5000909103010E946C190E94A80F2FEF81EE61
:100D600094E0215080409040E1F700C0000067E42B
:100D7000DDCF8CEF8C0F813AD0F46C2F8091020183
:100D8000909103010E94CA18882349F06C2F80912A
:100D90000201909103010E9477190E94A80F6C2F05
:100DA00080910201909103010E946C19C5CF80E2ED
:100DB0008C0F883048F4C77081E001C0880FCA9555
:100DC000EAF70E94690FB8CFEBE5EC0FE33040F48F
:100DD000F0E0E15CFE4F808190E0CF910C948818A8
:100DE000C85AC73158F4EC2FF0E0EE0FFF1FEF5E4A
:100DF000FE4F80819181CF910C949E18CF910895E0
:100E0000882309F45BC0682F823879F40E94271880
:100E100081FF54C069E380910201909103010E9417
:100E20006C190E94A80F69E310C08338B1F40E94C6
:100E3000271880FF43C063E5809102019091030170
:100E40000E946C190E94A80F63E5809102019091A5
:100E500003010E9477190C94A80F843879F40E943A
:100E6000271882FF2BC067E4809102019091030153
:100E70000E946C190E94A80F67E4E7CF8CEF860FE1
:100E8000813A18F380E2860F883048F4677081E079
:100E900001C0880F6A95EAF70E946F0FDCCF8BE5DF
:100EA000860F833020F480E090E00C948818685A14
:100EB000673120F480E090E00C949E1808951F9311
:100EC000CF93DF93182FEB010E945E06209741F02D
:100ED0008FE99FE00197F1F700C000002197F6CF5E
:100EE000812FDF91CF911F910C940007893319F066
:100EF00060E070E002C060E570E00C945F0788235A
:100F000021F00E94690F0C94A80F0895882321F006
:100F10000E946F0F0C94A80F0895CF92DF92EF926A
:100F2000FF920F931F93CF93DF937C01D62FC72F90
:100F3000FC011281058102950F700E945F0F8823CA
:100F4000B9F01123A9F08C2F807F803421F080E24A
:100F50008D0F883068F08091810282FD09C082E0A7
:100F60000E9408100E945F0F91E0D82ED92601C080
:100F7000D12CCC2EC2948FE0C8228C2D90E08C30E6
:100F8000910508F0C4C1FC01EA5AFF4F0C942D22D0
:100F90008C2F807FCF70882311F0C295C07F1123E2
:100FA00099F0CC2309F49FC180E28D0F883010F0B6
:100FB000D11104C08C2F0E94690F03C08C2F0E9496
:100FC000790F0E94A80F8FC18D2F0E940007CC239C
:100FD00009F49DC180E28D0F883038F1DD2329F1BD
:100FE0008C2F0E947F0F24C08C2F807FCF70803287
:100FF00011F0C295C07FDD2319F0D130A1F13DC0C1
:101000008091810282FF17C0112349F0CC2329F07F
:101010008C2F0E94690F0E94A80F80E065C180E0BC
:101020000E940007CC2309F472C18C2F0E946F0F1D
:101030000E94A80F6CC1112371F0002341F0013010
:1010400031F40E94890F8C2B0E94910F60C10E9485
:10105000890F8C2B1DC0002319F0013009F457C1F2
:101060000E949E0F25C0112321F0063008F04FC1C9
:101070000EC0053008F04BC11BC0112361F00023E6
:1010800031F0F701858180FF2EC18F7085838C2F11
:101090000E947F073CC1002359F0D93309F034C1C5
:1010A000FFEF07EE13E0F15000401040E1F72AC1D6
:1010B0008C2F0E9486072BC18C2F86958695837076
:1010C00019F0813061F023C1112321F08D2F9C2F65
:1010D000937002C080E090E00E94881820C1112324
:1010E00021F08D2F9C2F937002C080E090E00E9431
:1010F0009E1815C18C2F837009F047C011110BC1C8
:101100002D2F229526952770220F220F6D2F6F709D
:10111000862F90E0A0E0B0E0022E04C0880F991F57
:10112000AA1FBB1F0A94D2F7D4FF10C04FE050E0B3
:1011300060E070E004C0440F551F661F771F2A95BA
:10114000D2F7409550956095709503C040E050E00F
:10115000BA01C695C695C3708A019B01082B192B4D
:101160002A2B3B2BC901B801C23049F058F4C130D9
:1011700019F00E947F0ACFC00E946D0ACCC00E9465
:10118000910AC9C00E946B0AC6C0112319F08C2FA6
:10119000817001C08695882309F4BDC02D2F22954A
:1011A00026952770220F220F6D2F6F70862F90E0EB
:1011B000A0E0B0E0022E04C0880F991FAA1FBB1F39
:1011C0000A94D2F7D4FF10C04FE050E060E070E026
:1011D00004C0440F551F661F771F2A95D2F740950C
:1011E00050956095709503C040E050E0BA01C695F7
:1011F000C695C3708A019B01082B192B2A2B3B2B08
:10120000C901B801C23049F058F4C13019F00E9448
:10121000440B81C00E94320B7EC00E94560B7BC0E3
:101220000E94A50A78C0CF70112339F08C2F0E943C
:10123000CB0A8D2F0E947F076EC08D2F0E948607DC
:101240008C2F0E94EC0A67C0D23F21F128F4D03FD6
:1012500041F0D13FC1F043C0D33F19F1D43F79F001
:101260003EC0112341F0053008F051C08C2F8F7122
:101270000E94110B4CC0063008F049C0F7CF809196
:10128000810282FF18C0112339F08C2F8F710E94C8
:10129000CB0A3DC01123C9F38C2F8F710E94EC0A39
:1012A00036C0112329F08C2F8F710E94B60A2FC0EF
:1012B0000E94B10A2CC0112349F0CF718C2F0E94DB
:1012C000CB0A63E08C2F0E94ED0F21C081E00E94C9
:1012D00008100230E0F082E00E94081018C01123CC
:1012E00031F0002391F28D2F0E945E0610C0002382
:1012F00099F2D93349F41FEF27EE33E01150204023
:101300003040E1F700C000008D2F0E94000788EFF9
:101310008C0D843020F40E9427180E94CC05DD201B
:10132000C9F00E945B0F80FD15C0F70112820E9478
:10133000550F0E94CB0AC7010E94CB090E94550F8E
:10134000DF91CF911F910F91FF90EF90DF90CF90A1
:101350000C94EC0ADF91CF911F910F91FF90EF90C9
:10136000DF90CF9008950F931F93CF93DF93EC01FD
:10137000688179818A810E940D0C8C010E94680B22
:101380000E94590AB801CE010E948D07DF91CF91CA
:101390001F910F910895CF93DF93EC01988189817C
:1013A0002B813C81232B31F08F3F31F481E09F3F33
:1013B00019F403C081E001C080E080FD1DC0CE01B2
:1013C0000E942605811110C00E945F0F8823A1F0A2
:1013D0008A81882389F08091810282FD0DC082E09C
:1013E000DF91CF910C940810CE010E94B309CE0179
:1013F000DF91CF910C949904DF91CF91089580E013
:1014000090E00E94881880E090E00E949E180E9460
:10141000860F0C94A80F80910201909103010E9405
:1014200082190C94FF090E94760F0C940B0A929576
:101430009F70963079F010F4925001C09A5092301B
:1014400068F4803F69F018F4883E40F409C0843F96
:1014500029F406C0883E20F0813F11F080E0089515
:1014600081E00895FC01808191810E94020C0E941C
:10147000170A0895CF93DF9300D000D01F92CDB705
:10148000DEB70F900F900F900F900F90DF91CF91DC
:101490000895CF93DF9300D000D000D0CDB7DEB752
:1014A00026960FB6F894DEBF0FBECDBFDF91CF9169
:1014B0000895089508950C945A0A0C945B0A0E94AA
:1014C0005D0A6093B8017093B9018093BA0190935B
:1014D000BB010C94FF090C945F0A0F931F930091BA
:1014E000B8011091B9012091BA013091BB01602B74
:1014F000712B822B932B1F910F910C945F0A0F93EA
:101500001F930091B8011091B9012091BA01309157
:10151000BB0160237123822393231F910F910C94AD
:101520005F0A0F931F930091B8011091B9012091A8
:10153000BA013091BB0160277127822793271F9141
:101540000F910C945F0A0C94E2030E94A30A60932B
:10155000B4017093B5018093B6019093B7010C94D8
:10156000FF0960E070E0CB010C94A50A0F931F9374
:1015700041E050E060E070E08A019B0104C0000F90
:10158000111F221F331F8A95D2F7C901B8011F917D
:101590000F910C94A50A0F931F9341E050E060E077
:1015A00070E004C0440F551F661F771F8A95D2F75D
:1015B0008091B4019091B501A091B601B091B701AD
:1015C0008A019B01082B192B2A2B3B2BC901B8013F
:1015D0001F910F910C94A50A0F931F9341E050E0C7
:1015E00060E070E004C0440F551F661F771F8A95A6
:1015F000D2F740955095609570958091B401909187
:10160000B501A091B601B091B7018A019B010823F1
:1016100019232A233B23C901B8011F910F910C9470
:10162000A50A0F931F9341E050E060E070E004C012
:10163000440F551F661F771F8A95D2F78091B4011A
:101640009091B501A091B601B091B7018A019B01BB
:10165000082719272A273B27C901B8011F910F9195
:101660000C94A50A0F931F930091B4011091B5013A
:101670002091B6013091B701602B712B822B932BF7
:101680001F910F910C94A50A0F931F930091B40121
:101690001091B5012091B6013091B70160237123FB
:1016A000822393231F910F910C94A50A0F931F93EC
:1016B0000091B4011091B5012091B6013091B701AC
:1016C00060277127822793271F910F910C94A50AF9
:1016D00008952CE0929F800D1124E82FE695E69561
:1016E000E695877051E001C0550F8A95EAF785E0CD
:1016F000E89FF0011124EA56FE4F20E030E070E050
:101700004081CB01022E02C0969587950A94E2F79C
:101710008170819584278523842781932F5F3F4F94
:101720002530310569F708952CE0929F800D112432
:10173000682F669566956695982F977085E0689FE7
:10174000B001112440E050E080E0FB01E40FF51F00
:10175000EA56FE4F208130E0092E02C036952795CB
:101760000A94E2F721703327042E01C0220F0A9455
:10177000EAF7822B4F5F5F4F4530510531F70895EF
:10178000BF92CF92DF92EF92FF920F931F93CF936E
:10179000DF938C01C090B401D090B501E090B60108
:1017A000F090B7018091B8019091B901A091BA0170
:1017B000B091BB01C82AD92AEA2AFB2ACFE1D0E09E
:1017C000D701C6010C2E04C0B695A79597958795AD
:1017D0000A94D2F780FD04C0219790F7B12C07C07E
:1017E000BC2EB8018C2F0E9410130197A9F38B2DEA
:1017F000DF91CF911F910F91FF90EF90DF90CF90ED
:10180000BF900895CF93DF93EC010E94C00BBE01FF
:101810000E941013DF91CF9108951F93CF93DF9310
:10182000EB0190919501992321F0CB010E94020CCC
:1018300013C0882349F0CB010E94C00B182F682FDA
:10184000CE010E94690B04C0CB010E94940B182F9B
:10185000BE01812F0E941013DF91CF911F91089537
:101860001F93CF93DF93C091BC0116E08091BD011F
:10187000C81799F0D0E01C9FF0011D9FF00D1124B6
:10188000E254FE4F40815181628173818481958150
:101890000E94490A2196C770E9CFDF91CF911F912D
:1018A00008954091EE015091EF016091F001709127
:1018B000F1018091F2019091F3010C94490AEF92A9
:1018C000FF920F931F93CF93DF938091F301829543
:1018D0008F7009F065C08091F001882309F460C021
:1018E0008091BC01F090BD011091EE010091EF01DB
:1018F0006091F1017091F20191E01F3F09F090E0D9
:10190000C0910001D0910101292F96E0E92E8F1599
:1019100009F446C06115710521F00F3F21F030E058
:1019200003C031E001C0322F90E030FD36C0E89EA8
:10193000F001E99EF00D1124DF01A254BE4F119673
:101940003C911197301329C03C91311326C0129657
:101950003C911297311121C013964D915C911497CF
:10196000461B570B4C175D07C0F48091F3018F7035
:1019700080618093F301ED53FE4F80818F70806111
:1019800080838EEE91E00E94CB09DF91CF911F9171
:101990000F91FF90EF900C94300C01968770B7CFA9
:1019A000DF91CF911F910F91FF90EF9008959F923B
:1019B000AF92BF92CF92DF92EF92FF920F931F935D
:1019C000CF93DF93CDB7DEB761970FB6F894DEBF44
:1019D0000FBECDBF8C0185E0F801DE011D960190A0
:1019E0000D928A95E1F7D8011296EC909091EE0154
:1019F000E091EF012091F1013091F20121153105C3
:101A000031F0EF3F31F481E09F3F19F403C081E0F2
:101A100001C080E0B82FB1709B2E80FD47C1D80176
:101A20004C9111965C9111971396AD90BC901497C0
:101A30008EEEC82E81E0D82EF090F001B501621B29
:101A4000730B2091000130910101FF2009F4D9C0EE
:101A50008091F3016217730708F095C0282F207F4B
:101A600009F052C05E1313C0491311C0FE2CE110DF
:101A70000EC08F7080618093F3010E94510CC601EB
:101A80000E94CB098091F301F80185834DC1AB28F9
:101A900031F05F3F31F481E04F3F19F403C081E042
:101AA00001C080E080FD03C081E08E2502C080E09F
:101AB00090E0F82FF170FF2E80FF1CC08091BC01D8
:101AC0002091BD0136E0821709F40BC190E0389FE8
:101AD000F001399FF00D1124E254FE4F618156133D
:101AE00006C06081461303C06281E61203C00196FE
:101AF0008770E9CFFE2CEE2009F416C18091F30126
:101B000081608093F30154C05E1306C0491304C082
:101B1000E11002C0F80199C0C8010E94320A88236E
:101B200061F1EE2051F12091F301822F82958F70A7
:101B300090E0029774F08091EE019091EF01988708
:101B40008F831986BB86AA862C87CE0107960E94B2
:101B5000CB0986E0F801AEEEB1E001900D928A95D6
:101B6000E1F70E945F0C0E94510C0AC05E1711F150
:101B7000C8010E94320A81112CC0C8010E94CB0901
:101B8000FF24F394D1C0282F207F81F77A2DB98AC2
:101B9000A88A6E2D89890E943A0A8EEE91E00E94F1
:101BA000CB0986E0D6011D928A95E9F70E94510C77
:101BB000F12CBAC04913DCCFE110DACFF8018583EC
:101BC000C8010E94CB0986E0D6011D928A95E9F7EB
:101BD000ABC0EE2091F22091F301822F82958F709D
:101BE00090E002970CF4B5CF8091EE019091EF0157
:101BF0009A8389831B82BD82AC822E83CE0101969B
:101C0000A6CF6217730708F044C0FE2CEE2009F43B
:101C1000B4CF5E1330C049132EC02091F30120FDD4
:101C200021C0822F82958F70482F50E041155105B9
:101C3000C9F0F80125834F30510541F08F5F982F8F
:101C40009295907F822F8F70892B8583C8010E9487
:101C5000CB0986E0F801AEEEB1E001900D928A95D5
:101C6000E1F73CC086E0F801AEEEB1E001900D92E4
:101C70008A95E1F759C0C8010E94320A811169CFE3
:101C80008091F30181608093F301C8010E94CB0928
:101C90004BC07A2DB98AA88A6E2D89890E943A0A8A
:101CA00086E0D6011D928A95E9F718C0EE2009F466
:101CB00064CFC8010E94320AF82E882309F45DCF50
:101CC00086E0F801AEEEB1E001900D928A95E1F761
:101CD0008EEE91E00E9458060E945F0C0E94510C0B
:101CE00023C04D875E878D859E850E94020C292F1B
:101CF00022952F70223028F49F7039F0811105C091
:101D00000BC0243028F49F7049F4805E883020F0A6
:101D1000C8010E94CB099F2CF92C06C0D80115964A
:101D20009C91907F91F7F8CF8F2D61960FB6F89424
:101D3000DEBF0FBECDBFDF91CF911F910F91FF90FE
:101D4000EF90DF90CF90BF90AF909F9008951F933A
:101D5000CF93DF93CDB7DEB72C970FB6F894DEBFE5
:101D60000FBECDBF4F83588769877A878B879C8743
:101D7000CE0107960E94D70C8823D1F09F818885D9
:101D80002A853B85232B31F08F3F31F481E09F3F43
:101D900019F403C081E001C080E080FD47C04F819D
:101DA000588569857A858B859C850E94490A3EC045
:101DB00086E0FE013796DE01119601900D928A951C
:101DC000E1F7FF81E8856A857B856115710531F052
:101DD000EF3F31F481E0FF3F19F403C081E001C01F
:101DE00080E080FD23C02091BD0130E0C901019653
:101DF000877099274091BC0150E084179507F1F155
:101E0000F983EA837D836C8396E0929FD001939F50
:101E1000B00D1124A254BE4FFE01319601900D92D7
:101E20009A95E1F78093BD010E94300C16E08091F5
:101E3000BC019091BD01891771F1189FC001112457
:101E400082549E4F0E94D70C882329F1E091BC0157
:101E50001E9FF0011124E254FE4F408151816281A6
:101E60007381848195810E94490A8091BC0190E030
:101E70000196877099278093BC01D9CF0E94130ADD
:101E80001092BD011092BC01EEEEF1E086E0DF01A0
:101E90001D928A95E9F72C960FB6F894DEBF0FBE17
:101EA000CDBFDF91CF911F91089580911402859548
:101EB0008595859508958091140287700895909175
:101EC0001402977081E009F480E008958091370250
:101ED000089590913702892B809337020895809559
:101EE0009091370289238093370208951092370228
:101EF000089590913602892B80933602089580953B
:101F0000909136028923809336020895109236020A
:101F1000089580911502089508950C948C0F0C94E7
:101F20008D0F9091810292FD08C090911502981733
:101F300021F0809315020C948F0F08958091150263
:101F4000882329F01092150280E00C948F0F0895D9
:101F5000CF93DF93E0910201F0910301809137026A
:101F60008083E0910201F09103019081809136021B
:101F7000892B808380911502882381F0E0910201F2
:101F8000F09103019081892B8083809102019091CF
:101F900003010E94B41881110E949E0FC09102019A
:101FA000D091030140E250E064EF71E0CE010E9465
:101FB0003322892B69F080E2FE01A4EFB1E00190A9
:101FC0000D928A95E1F7CE01DF91CF910C943318F1
:101FD000DF91CF9108950C948C0F9091810292FD26
:101FE00010C098E0899F90011124262B20931402A1
:101FF0000E94CB0A809114028595859585950C9455
:10200000EB0F0C94CB0A1092140280E00C94EB0FAF
:10201000209114028095822380931402982F977048
:1020200099F430E0482F082E000C550B2417350783
:1020300059F09091810292FD07C08595859585950F
:102040000E94EC0A0C9403100895CF9390918102A2
:1020500092FB222720F92817F9F0C82F892FC0FBFF
:1020600082F98093810280918002909181020E9486
:102070008C1082E00E9408108091480280FF0CC002
:102080001F92CF9385EE93E09F938F930E94D50389
:102090000F900F900F900F90CF9108958091810233
:1020A00082FB882780F991E089270C94251081E034
:1020B0000C94251080E00C9425106FEF7FEF80E0EA
:1020C00090E00C946C2280E090E00E94482221E095
:1020D000893E9E4F09F020E0822F089582E090E033
:1020E0000C94402283E090E00C944022682F83E01F
:1020F00090E00C944E22CF9384E090E00E94402226
:10210000C82F82E290E00E9440222C2F30E0A901EB
:10211000582BCA01CF910895CF93C92F682F84E01F
:1021200090E00E944E226C2F82E290E0CF910C94BE
:102130004E22AB01BC018FE090E00C946022AB0119
:10214000BC0183E190E00C94602260E070E0CB0180
:102150000C949F1060E070E0CB010E9499100C94E9
:10216000A51069EE7EEF80E090E00E946C2260E0B6
:1021700082E090E00E944E2260E083E090E00E94C6
:102180004E221092B8011092B9011092BA01109229
:10219000BB0160E084E090E00E944E2260E082E2B9
:1021A00090E00E944E2260E085E090E00E944E2286
:1021B00060E086E090E00E944E226FEF87E090E0C2
:1021C0000E944E2240E050E0BA0188E090E00E9478
:1021D000602260E08DE090E00E944E2240E050E0FE
:1021E000BA0188E190E00E94602260E087E190E01F
:1021F0000E944E2240E050E0BA018CE190E00E9443
:10220000602260E070E080E290E00E946C2240E09A
:1022100050E0BA0188E190E00E9460220C94AA107C
:102220000C94B110682F8EE090E00C944E220E9426
:102230003C1A609344027093450280934602909347
:102240004702609340027093410280934202909350
:102250004302089585B7806885BF85B7806885BFCC
:10226000089581E008950C94311108950C9435116E
:102270000C9435110C9438110C9435110C943C11BC
:102280000C9435110E942A118BE69CE10E941D18C6
:102290000E9440110C943E110E9436110C9435118D
:1022A0000E9404140C94CB050E94271A0E942B153F
:1022B0000E9450110C943A115F926F927F928F920C
:1022C0009F92AF92BF92CF92DF92EF92FF920F93C5
:1022D0001F93CF93DF93CDB7DEB72A970FB6F8944D
:1022E000DEBF0FBECDBF0E944015C82E81110E94D7
:1022F000171138E3832E32E0932E00E010E0502EC9
:10230000802F0E9428145C01F401619071904F01AC
:102310006826792661147104B1F40F5F1F4F0430F1
:10232000110569F78FEF89838A831B820E94301A17
:102330008160782F9D838C8349815A816B818D8147
:102340000E940E063AC08091480281FD0E9431141D
:10235000D12CEE24E394F12CC3018E219F21892BF3
:1023600029F10E9433118823A9F0DE825F82AE201A
:10237000BF2081E0AB2809F480E088870E94301AF2
:102380008160782F9A8789874E815F8168858A85E9
:102390000E940E06000F111FF801E85CFD4F8081BE
:1023A0009181E826F926F182E08207C0D394EE0CF1
:1023B000FF1CFCE0DF12D0CFB0CF81E0C11001C024
:1023C00080E02A960FB6F894DEBF0FBECDBFDF9136
:1023D000CF911F910F91FF90EF90DF90CF90BF9022
:1023E000AF909F908F907F906F905F9008950E9424
:1023F0005C110C94DC05CF93DF930E941513EC0164
:10240000811522E59207E8F5811531E5930708F07B
:10241000B6C0883E910528F5803E910508F0E9C0D8
:10242000883A910570F4853A910508F07AC08130B8
:10243000910509F473C008F4D9C0049708F0D9C015
:10244000D5C08F3B910508F0D1C0C85AD0E0CC0F61
:10245000DD1FCE5BDE4F0990D881C02DCE01946484
:10246000C9C0811540E5940708F069C0811550E4A2
:10247000950708F060C09A9581159F4108F4B9C08E
:10248000B5C0811536E5930728F5811545E5940714
:1024900008F092C0811554E5950708F087C0AC019B
:1024A00043705527282F26952695C115D34508F04A
:1024B0006CC081E090E002C0880F991F4A95E2F756
:1024C00040E2249F90011124EC01C22BD32BCE01BA
:1024D0009C6890C081152AE5920780F4811539E542
:1024E000930708F072C0811548E5940708F47EC090
:1024F000D82FCC27CE01806F906A7CC09056811572
:10250000904208F073C08D2F8F710E94A913DD27B0
:10251000D0628F71AE01582BCA016CC081E090E08F
:1025200069C0C55AD0E0C059DE4F8881C82FD0E0BD
:10253000CE0190645FC0DF70CE01906A5BC074E032
:10254000969587957A95E1F7282F23703C2F337065
:1025500081E090E002C0880F991F3A95E2F79C68ED
:10256000AC01522B9A019C2F9F709695969550E244
:10257000959FE0011124C9018C2B9D2B3BC0D82FC6
:10258000CC27CE01816F906A35C081E090E002C017
:10259000880F991F4A95E2F750E2259F9001112478
:1025A000EC01C22BD32BCE019A6824C0D82FCC27A4
:1025B000CE01846F906A1EC00E94A9138F7190E0B3
:1025C000D82FCC27CE01906215C08F700E94A9131E
:1025D00094E0D695C7959A95E1F7CF70D0E0DC2FBF
:1025E000CC27D0699E01282BC90104C080E090E06F
:1025F00001C0CE01DF91CF91089520E3829FC001F9
:102600001124FC012CE0729FE00DF11D1124E60F56
:10261000F11DEE0FFF1FE05FFE4F8591949108952D
:102620000E94FD120E94FB1108958238910569F104
:10263000B0F48133910509F46DC048F489329105F5
:1026400009F463C08A32910509F469C0089585339D
:10265000910509F455C089339105B9F00895833E79
:10266000910569F138F4803E9105B1F0823E910503
:1026700009F10895863E9105A9F1873E9105B9F1CA
:10268000843E910509F064C023C02091800220FDA2
:102690004FC021FD4DC008958091800280FD44C04F
:1026A0008091810280FF44C08091800284FD42C0FD
:1026B00083EE4DC08091800282FF38C0F5CF8091BB
:1026C000800282FD33C08091810280FD31C0ECCF59
:1026D0008091810281FF32C08091800284FD2AC0F6
:1026E00087EE35C08091800283FF26C0F5CF8091B0
:1026F000800283FD21C08091810281FD1FC0ECCF4B
:102700008091800285FD1CC01DC08091800285FDE6
:1027100019C016C08091800286FD16C017C0809136
:10272000800286FD13C010C089E311C082EE0FC085
:1027300080EE0DC080E00BC086EE09C084EE07C0BD
:1027400089E205C085E303C08AE201C081E390E02D
:1027500008959091800292FF0DC0282F2871283093
:1027600019F4877F846006C0282F2471243011F467
:102770008B7F886093FF0DC0282F2871283119F4B2
:10278000877E846106C0282F2471243111F48B7E4A
:1027900088612091810220FF0DC0382F38713830B8
:1027A00019F4877F816006C0382F3171313011F400
:1027B0008E7F886021FF0DC0282F2871283119F4E1
:1027C000877E816106C0282F2171213111F48E7E10
:1027D000886194FD877E08950C945D100E944015D9
:1027E0008FE39CE90197F1F700C000000E944015BB
:1027F00080E00E94281480FF04C00E94EC130C9417
:102800007D1A08950C94EE130E946310811102C08A
:102810000E9410110E946E10809348020E947B104B
:1028200090938102809380020E9402140E94721091
:10283000682F70E080E090E00E946B0A6091B40124
:102840007091B5018091B6019091B7010C94A30AE3
:10285000E82FF0E0EE0FFF1FE657FD4F80819181DA
:102860000895CF92DF92EF92FF920F931F93CF9331
:10287000DF938AE094E00E943C038AE8E82E82E03D
:10288000F82EC0E0D0E095E0C92E94E0D92E0CEFF0
:1028900013E0DF93CF93DF92CF920E94D50382E0C3
:1028A00094E00E943C03F701819191917F010E9485
:1028B000B1059F938F931F930F930E94D5038AEFC7
:1028C00093E00E943C0321968DB79EB708960FB601
:1028D000F8949EBF0FBE8DBFC430D105D1F6DF91F5
:1028E000CF911F910F91FF90EF90DF90CF900895BF
:1028F00080EA8A95F1F7089500C008950C94781441
:1029000008950C9453040C948014F894E82FE295E5
:10291000EF70F0E031A1282F2F7081E090E001C02E
:10292000880F2A95EAF7982F9095932391A392A167
:10293000892B82A3789408950F931F93CF93DF93ED
:10294000CFE7D1E089918F3F11F00E94851481E09B
:10295000C338D807B9F7C3E7D1E00FE711E0899191
:102960008F3F11F00E9485140C171D07C1F7DF91EE
:10297000CF911F910F910895BF92CF92DF92EF9266
:10298000FF920F931F93CF93DF938C01C62FD0E05C
:10299000CE0181589E4F6C01FC0190819F3F09F44C
:1029A00050C0B62EF894E92FE295EF70F0E081A1C7
:1029B0009F7021E030E001C0220F9A95EAF7822B48
:1029C00081A382A12095282322A378940E947C14BD
:1029D000E3E7F1E04FE751E021E030E0E12CF12CBA
:1029E00061916F3F89F0A62FA295AF70B0E09096ED
:1029F0008C9190E06F7002C0959587956A95E2F78B
:102A000080FD02C0C90102C080E090E0E82AF92AF6
:102A1000220F331F4E175F0719F7F60180818F3F92
:102A200011F00E94851461E0E114F10409F460E002
:102A30008B2D0E947E14CC0FDD1FC00FD11FF98299
:102A4000E882DF91CF911F910F91FF90EF90DF907F
:102A5000CF90BF9008950E949C1488E0EAE8F2E0CD
:102A6000DF01982F1D929A95E9F7E2E8F2E0DF0185
:102A70001D928A95E9F784E00E948B150C9412054B
:102A8000FF920F931F93CF93DF93CDB7DEB72897B5
:102A90000FB6F894DEBF0FBECDBF8E010F5F1F4F84
:102AA00088E0F80111928A95E9F7F12C6F2DC801A1
:102AB0000E94BC14F394F4E0FF12F8CF48E050E019
:102AC000B80182E892E00E943322FF24F394009739
:102AD00009F4F12C892B41F088E0F801A2E8B2E07A
:102AE00001900D928A95E1F72F2D44E06AE872E09B
:102AF00082E892E00E948C150E9414058F2D289682
:102B00000FB6F894DEBF0FBECDBFDF91CF911F91FE
:102B10000F91FF9008950895FF920F931F93CF9305
:102B2000DF93F82E092F162FD72FC42F222349F019
:102B300081E080934B020E94301A90934A02809366
:102B4000490280914B028823D9F0809149029091EB
:102B50004A020E94481A059798F0EF2DF02FA12FF6
:102B6000BD2F80E090E04C2F50E08417950734F49F
:102B7000219131912D933D930196F7CF10924B0205
:102B8000DF91CF911F910F91FF9008950E94E71C54
:102B90000E9454110C94F31C0E94F71C0E94F71120
:102BA0000C94151D0E94CE190E94CE1C0E94421149
:102BB0000E94C6150E94CC150E944C11FBCFCF93EA
:102BC000DF93EC01FB018281882309F43CC1C4300E
:102BD000FDE5DF0760F4CB3F9CE5D90788F49E0153
:102BE00022503C452431310508F02EC109C0C236BF
:102BF000EDE5DE0729F0C63AFDE5DF0709F024C15F
:102C00000E947B109093810280938002C1318CE5F9
:102C1000D80709F4C6C008F042C0C930ECE5DE07A9
:102C200009F49BC000F5C5308CE5D80709F485C0D0
:102C300078F4C330ECE5DE0709F478C008F07AC018
:102C4000C230DC4509F0F5C0809180028160EFC0A0
:102C5000C7309CE5D90709F478C008F07AC08091A4
:102C600080028061E4C0CD30FCE5DF0709F487C055
:102C700058F4CB309CE5D90709F479C008F07BC043
:102C80008091800288606FC0CF30FCE5DF0709F4D7
:102C900080C008F082C080918002877FC8C0CE3F8C
:102CA0009CE5D90709F471C000F5C531FCE5DF07E3
:102CB00009F485C068F4C3319CE5D90709F475C0EF
:102CC00008F095C00E94130A809180028F77AFC0F0
:102CD000CC3FFCE5DF07A9F108F054C0CB3FDC4551
:102CE00009F0A7C08091810240C0C230EDE5DE0747
:102CF00009F489C058F4C1158DE5D80709F45AC004
:102D000008F069C08091810282602FC0C236EDE573
:102D1000DE0709F47CC0C63AFDE5DF0709F481C08F
:102D2000C330DD4509F085C080E06EC0809180022F
:102D300082607DC08091800216C080918002886090
:102D400076C08091810282604FC080918002806253
:102D50006EC08091800280646AC00E94130A8091D4
:102D60008002806864C0846062C081603DC08091E0
:102D700080028E7F5CC0809180028D7F58C08091E0
:102D8000800216C08091810218C0809181028D7FDF
:102D90002BC0809180028F7E4AC0809180028F7DFF
:102DA00046C0809180028F7B42C080918002877FE5
:102DB0008B7F3DC0809181028D7F8E7F15C0809179
:102DC000800282FB222720F991E0922790FB82F972
:102DD00090FB83F92CC080918102982F909591707F
:102DE0008E7F892B90FB81F98093810222C00E9403
:102DF000130A8091800287FB222720F991E0922715
:102E000090FB87F914C081E00E94121112C08091DA
:102E1000800284FB222720F991E0922790FB84F91D
:102E200006C080918002982F909590FB80F9809346
:102E3000800280918002909181020E948C100E94F9
:102E4000130A80E001C081E0DF91CF910895CF9314
:102E5000DF9386319C4541F5EB010E94660F982F68
:102E60008A812091020130910301882379F09A7AB6
:102E700081E009F480E080934C02911102C069E284
:102E800001C065E3C9010E946C190AC080914C021F
:102E9000811102C069E201C065E3C9010E9477198E
:102EA0000E94A80F80E001C081E0DF91CF910895DA
:102EB0000F931F93CF93DF93C42FD22FFC018281F6
:102EC0008823C9F040934F020E94301A90934E021B
:102ED00080934D0280E28C0F883008F057C0C77095
:102EE00081E001C0880FCA95EAF7DF91CF911F9169
:102EF0000F910C947F0780914F02481330C080914E
:102F00004D0290914E020E94481A883C910538F576
:102F100010E21D0FCD17B9F080E28C0F883040F41D
:102F2000C77081E001C0880FCA95EAF70E94860742
:102F3000183028F581E09D2F977001C0880F9A9571
:102F4000EAF70E947F07802F0E9476071830F0F47E
:102F5000D77081E001C0880FDA95EAF70AC080E2F5
:102F60008C0F883098F4C77081E001C0880FCA9533
:102F7000EAF7DF91CF911F910F910C948607802F74
:102F8000DF91CF911F910F910C947607DF91CF9134
:102F90001F910F9108950F939C01CB01243F4CE5A5
:102FA000340731F188F4293DFCE53F07D9F02A3D8B
:102FB0004CE5340779F1283D3C45A9F506E221EEC0
:102FC00041EE68ED7CE52BC0263FFCE53F07E1F0D4
:102FD000A8F0273F3C4539F507E225EE46EE67EFBE
:102FE0007CE51DC007E225EE45EE69ED7CE517C0E6
:102FF00006E221EE40EE64EF7CE511C007E225EE2B
:1030000044EE65EF7CE50BC006E221EE42EE66EF92
:103010007CE505C008E221E045EE6AED7CE50E9412
:10302000581780E008C0FC018281882319F01092B3
:103030004F0201C081E00F91089590939301809316
:103040009201089590935502809354020895E0915F
:103050005402F0915502309721F00190F081E02D5B
:10306000099480E00895EF92FF921F93CF93DF932E
:10307000FC01A0915402B0915502109709F442C08E
:1030800080911001882341F08091800287FF04C065
:103090008081818386E08083EF011296ED91FC911F
:1030A0001397CE0109958091480282FF2BC080FFC3
:1030B00004C089E294E00E943C0318E083E2E82E19
:1030C00084E0F82E8091480280FF0BC088811F9217
:1030D0008F93FF92EF920E94D5030F900F900F9065
:1030E0000F90115021961111EDCF8091480280FF71
:1030F00009C081E294E0DF91CF911F91FF90EF90A2
:103100000C943C03DF91CF911F91FF90EF900895B5
:1031100020915202309153022817390771F0909391
:10312000530280935202E0915402F091550230977D
:1031300021F00680F781E02D099408952091500236
:10314000309151022817390771F090935102809302
:103150005002E0915402F0915502309721F0008422
:10316000F185E02D09940895FC01329680911001BB
:10317000882331F08091800287FF02C09EE101C068
:1031800096E080E0915028F021912223D9F38F5FBF
:10319000F9CF0895662351F1209110012223E9F01F
:1031A0002091800227FF19C0462F469546954695E7
:1031B0004E31E0F4677021E030E002C0220F331F8F
:1031C0006A95E2F7FC01E40FF11D828190E028236B
:1031D000392381E0232B69F409C0FC01329608965B
:1031E0002191621729F0E817F907D1F780E00895D7
:1031F00081E008959C01FC0132969FEF80E04191AF
:10320000461789F09F3F19F4411101C0982F8F5F35
:103210008630A9F79F3F39F0F901E90FF11D97FDBD
:10322000FA956283089508959C012A5F3F4FFC013F
:103230004281461301C01282019682179307B9F7A3
:103240000895262F2695269526952E3170F4FC019B
:10325000E20FF11D677021E030E001C0220F6A9596
:10326000EAF78281282B228308958091480280FF0B
:103270000CC01F926F9389E594E09F938F930E94F7
:10328000D5030F900F900F900F900895262F26953D
:10329000269526952E3178F4FC01E20FF11D67701A
:1032A00021E030E001C0220F6A95EAF72095828183
:1032B0002823228308958091480280FF0CC01F922A
:1032C0006F938BE394E09F938F930E94D5030F90AD
:1032D0000F900F900F90089520911001222329F054
:1032E0002091800227FD0C9421190C94FA1820914A
:1032F0001001222329F02091800227FD0C94461909
:103300000C94141920911001FC013296222331F003
:103310008091800287FF02C08EE101C086E0DF015C
:103320001D928A95E9F7089508950C94941983E005
:10333000809356020C949519811102C081E001C05E
:1033400082E0809356020C9495190C949C1981E0AC
:10335000809356020C9495190C94A71908950C9417
:10336000AE190C94AF190C94AE190C94AE190C94C0
:10337000AE19CF930E94B5190E9440150E94B3194F
:10338000C0E08C2F0E942814892B29F4CF5FC43011
:10339000C1F780E001C081E0CF91089508951F92A8
:1033A0000F920FB60F9211248F939F93AF93BF93F9
:1033B00080915702811113C08091920290919302E3
:1033C000A0919402B09195024196A11DB11D8093E8
:1033D000920290939302A0939402B0939502BF91AE
:1033E000AF919F918F910F900FBE0F901F901895E6
:1033F00080919A02843031F10E9497051092570211
:1034000020E488E190E00FB6F894A89580936000DE
:103410000FBE2093600083B7817F846083BF83B732
:10342000816083BF7894889583B78E7F83BF0FB602
:10343000F894A89580916000886180936000109254
:1034400060000FBE08950E94130A0C949B0582E051
:1034500084BD93E095BD9AEF97BD80936E0008956B
:103460002FB7F8948091920290919302A0919402C8
:10347000B09195022FBF08952FB7F89460919202F2
:103480007091930280919402909195022FBF0895BC
:103490009C014FB7F8948091920290919302A09171
:1034A0009402B09195024FBF821B930B08957894BC
:1034B0001F920F920FB60F9211248F939F93AF9389
:1034C000BF938091920290919302A0919402B09147
:1034D00095020196A11DB11D8093920290939302D3
:1034E000A0939402B0939502BF91AF919F918F9159
:1034F0000F900FBE0F901F90189581E08093E00011
:1035000080E28093D8001092C9008FE19EE4019779
:10351000F1F700C0000087E090EBDC018093A3028C
:103520009093A402A093A502B093A6029CE088E128
:103530000FB6F894A895809360000FBE909360003A
:10354000FFCF80917E0208950895CF93DF9320915D
:103550001001222339F02091800227FF03C060E28E
:1035600022E002C068E021E02093E9002FEF3091D3
:10357000E800215035FD06C035ED3A95F1F7000021
:103580002111F5CF2091E80025FF1DC0EC018091AD
:103590001001811105C040E050E068E070E003C018
:1035A00070E040E050E0CE010E94841D8091E80070
:1035B0008E778093E80080E2FE01AEE5B2E00190F4
:1035C0000D928A95E1F7DF91CF91089580935A0289
:1035D00070935C0260935B0280919A02843001F5E3
:1035E00082E08093E9008FEF9091E800815095FD93
:1035F00006C095ED9A95F1F700008111F5CF809105
:10360000E80085FF0DC040E050E063E070E08AE52F
:1036100092E00E94841D8091E8008E778093E800FC
:103620000895BC0184E00C94E61ABC0183E00C947C
:10363000E61A08958BE894E00E943C038091990279
:10364000811109C00E94151F0E94721F8091E20023
:1036500084608093E200089587E894E00E943C0330
:1036600010929902089583E894E00E943C030C9420
:10367000AC198FE794E00E943C036091960281E0D0
:10368000611101C080E00C9497198BE794E00E94CF
:103690003C0390919A0281E0943009F080E06091BF
:1036A00096020C949C19209159022F5F822F62E39D
:1036B0000E942122992319F0209359020895109213
:1036C000590280915D02882371F180919A028430C1
:1036D00041F58091E9008F702091EC00922F91705C
:1036E00020FD90E8892B93E09093E9009091EB0006
:1036F00090FF14C09091EE0097FF10C09091E800E9
:1037000095FF03C01092F100F9CF9091E80090FF6F
:1037100005C09091E8009E779093E8008F708093A9
:10372000E90010925D02089542E061EC81E00E94A0
:103730008E1E42E261EC82E00E948E1E42E261EC4B
:1037400083E00E948E1E90919A0281E0943009F0ED
:1037500080E0609196020C94A51980919C028330C0
:1037600009F461C030F4813071F0823009F49AC0FC
:1037700008958A3009F486C08B3009F46CC0893012
:1037800009F0A8C020C080919B02813A09F0A2C034
:103790008091E800877F8093E80080919F0290915C
:1037A000A002892B21F460E28EE592E003C060E084
:1037B00080E090E070E00E94CF1D8091E8008B7760
:1037C0008093E800089580919B02813209F082C0C5
:1037D00080919F029091A002029708F07BC0809197
:1037E000E800877F8093E8008091E80082FD05C0B3
:1037F00080919A028111F8CF6DC02091F3008091E1
:10380000F20090E0922B029731F48091F100813028
:1038100011F0863021F48091F10080937E02809136
:10382000E8008B7753C080919B02813A09F052C027
:1038300080919F029091A002892B09F04BC080914A
:10384000E800877F8093E8008091E80080FFFCCF4C
:103850008091100136C080919B028132D9F5809110
:103860009F029091A002892BA9F58091E800877FA3
:103870008093E8000E94C31E80919D0280931001F6
:103880000C94130A80919B02813221F58091E8000B
:10389000877F8093E8000E94C31E80919E028093E0
:1038A0007F02089580919B02813AA1F48091E80003
:1038B000877F8093E8008091E80080FFFCCF8091B3
:1038C0007F028093F1008091E8008E778093E8007A
:1038D0000C94C31E08959FB7F89410925D029FBF89
:1038E00090919A02943009F057C09091E9009F702E
:1038F0003091EC00232F217030FD20E8922B23E043
:103900002093E9002091EB0020FF43C02091EE00BE
:1039100027FF3FC020915802222321F02091E80088
:1039200025FF37C01092580226E03091E80035FD9F
:1039300015C030919A02343061F53091EB0035FDBD
:1039400028C0215021F481E08093580222C0EFE981
:10395000FFE03197F1F700C00000E7CF8093F1005E
:103960008091E80085FD0AC08091E80080FFFCCFCF
:103970008091E8008E778093E80006C08FB7F894B6
:1039800021E020935D028FBF9F709093E90080E05B
:1039900008959F709093E9008FEF089584B7877F13
:1039A00084BF0FB6F894A8958091600088618093D9
:1039B0006000109260000FBE90E080E80FB6F894AF
:1039C00080936100909361000FBE0C94A7190E9430
:1039D000151F0E94721FE2EEF0E0808184608083F8
:1039E00078940C94062284E091E00C942218809143
:1039F0009A028530C9F487E794E00E943C038091E5
:103A00009A02853079F40E94F819809198028823EF
:103A1000B1F30E94B919882391F30E946E1D0E9490
:103A2000130AEDCF0C94231A089508950C94181DD1
:103A3000292F332723303105C9F060F421303105B7
:103A400081F02230310509F041C08BE590E02FEA8A
:103A500034E040C021323105E1F02232310531F14C
:103A600035C082E190E02AE035E034C0992781300A
:103A7000910549F028F0029749F5EFE8F4E005C018
:103A8000EBEAF4E002C0EFE9F4E0849190E09F01FA
:103A900021C063307105D0F4660F771FFB01E45736
:103AA000FE4F2081318189E090E014C063307105C0
:103AB00068F4FB01EE0FFF1FEA57FE4F20813181B2
:103AC000FB01ED57FE4F808190E004C080E090E064
:103AD00020E030E0FA0131832083089580E189BD40
:103AE00082E189BD09B400FEFDCF8091D8008F7DB1
:103AF0008093D8008091E00082608093E000809104
:103B0000E00081FDFCCF0895CF92DF92EF92FF920B
:103B10000F931F93CF93DF93EC018B017A010E94E7
:103B2000E21E811133C0E114F10439F0F701808104
:103B30009181081B190BC80FD91FC12CD12C01155D
:103B4000110519F18091E80085FD16C08091E8000B
:103B50008E778093E800E114F10449F0F701808149
:103B60009181C80ED91ED182C08285E00FC00E940B
:103B7000E21E882321F30AC089918093F10001504D
:103B80001109FFEFCF1ADF0ADACF80E0DF91CF9182
:103B90001F910F91FF90EF90DF90CF9008952091AB
:103BA000A1023091A2022617370748F0611571056E
:103BB00039F42091E8002E772093E80001C0B90184
:103BC000FC0120E06115710579F180919A0288234A
:103BD000F1F18530F1F18091E80083FD3CC08091E6
:103BE000E80082FD2EC08091E80080FFEBCF20919D
:103BF000F3008091F20090E0922B6115710551F075
:103C00008830910538F421912093F10061507109B9
:103C10000196F3CF21E0089709F020E08091E800B9
:103C20008E778093E800CECF2111CFCF0AC080914C
:103C30009A02882361F0853061F08091E80083FD6D
:103C40000AC08091E80082FFF2CF80E0089582E010
:103C5000089583E0089581E008952091A1023091B4
:103C6000A2022617370748F06115710539F4209133
:103C7000E8002E772093E80001C0B901FC0120E0A4
:103C80006115710591F180919A02882309F440C071
:103C9000853009F43FC08091E80083FD3DC08091EC
:103CA000E80082FD2FC08091E80080FFE9CF2091DD
:103CB000F3008091F20090E0922B6115710559F0AC
:103CC0008830910540F424912093F10031966150A1
:103CD00071090196F2CF21E0089709F020E0809168
:103CE000E8008E778093E800CBCF2111CCCF0AC0BB
:103CF00080919A02882361F0853061F08091E8001C
:103D000083FD0AC08091E80082FFF2CF80E0089531
:103D100082E0089583E0089581E00895982F973018
:103D200068F59093E900981739F07091EC002091B4
:103D3000ED005091F00003C0242F762F50E021FDBC
:103D400002C09F5FECCF3091EB003E7F3093EB00E1
:103D50003091ED003D7F3093ED003091EB0031600C
:103D60003093EB007093EC002093ED005093F00043
:103D70002091EE0027FDE5CF80E008958F708093BD
:103D8000E90081E0089580919B0287FF11C0809136
:103D9000E80082FD05C080919A028111F8CF11C020
:103DA0008091E8008B770BC080919A02882349F0BC
:103DB0008091E80080FFF8CF8091E8008E778093B3
:103DC000E80008952091E4003091E50095E64091E7
:103DD000EC00842F817040FF23C08091E80080FDBB
:103DE0001DC080919A02882399F0853099F08091C6
:103DF000EB0085FD11C04091E4005091E5002417CF
:103E0000350729F3915011F09A01E1CF84E008952C
:103E100082E0089583E0089581E0089580E00895A8
:103E20004091E80042FFDDCF08950E94831F0E9469
:103E30008B1FE0EEF0E0808181608083E8EDF0E0B0
:103E400080818F77808319BCA7EDB0E08C918E7F45
:103E50008C9380818F7E80831092990208950F93B6
:103E60001F93CF93DF930E94831F0E948B1FC8ED87
:103E7000D0E088818F778883888180688883888173
:103E80008F7D888319BC10929A021092960210922C
:103E900098021092970200EE10E0F80180818B7F6B
:103EA000808388818160888342E060E080E00E94B6
:103EB0008E1EE1EEF0E080818E7F8083E2EEF0E006
:103EC000808181608083808188608083F801808127
:103ED0008E7F8083888180618883DF91CF911F915D
:103EE0000F910895E8EDF0E080818F7E8083E7ED0B
:103EF000F0E080818160808384E082BF81E08093F4
:103F000099020C942F1FE8EDF0E080818E7F808372
:103F10001092E20008951092DA001092E1000895E4
:103F20001F920F920FB60F9211242F933F934F932E
:103F30005F936F937F938F939F93AF93BF93EF9311
:103F4000FF938091E10082FF0BC08091E20082FF2D
:103F500007C08091E1008B7F8093E1000E94531B9A
:103F60008091DA0080FF1FC08091D80080FF1BC0C5
:103F70008091DA008E7F8093DA008091D90080FFF3
:103F80000DC080E189BD82E189BD09B400FEFDCF8D
:103F900081E080939A020E941A1B05C019BC1092FE
:103FA0009A020E942C1B8091E10080FF19C0809131
:103FB000E20080FF15C08091E2008E7F8093E200D6
:103FC0008091E20080618093E2008091D80080625D
:103FD0008093D80019BC85E080939A020E94391B17
:103FE0008091E10084FF30C08091E20084FF2CC00A
:103FF00080E189BD82E189BD09B400FEFDCF8091D9
:10400000D8008F7D8093D8008091E1008F7E8093CF
:10401000E1008091E2008F7E8093E2008091E200D7
:1040200081608093E20080919602882311F084E001
:1040300007C08091E30087FD02C081E001C083E0FA
:1040400080939A020E94451B8091E10083FF29C062
:104050008091E20083FF25C08091E100877F8093FB
:10406000E10082E080939A02109296028091E10032
:104070008E7F8093E1008091E2008E7F8093E2004A
:104080008091E20080618093E20042E060E080E0A5
:104090000E948E1E8091F00088608093F0000E9444
:1040A000331BFF91EF91BF91AF919F918F917F91C2
:1040B0006F915F914F913F912F910F900FBE0F9095
:1040C0001F9018951F920F920FB60F9211242F93E5
:1040D0003F934F935F936F937F938F939F93AF9390
:1040E000BF93CF93DF93EF93FF93C091E900CF701D
:1040F0008091EC00D82FD17080FDD0E81092E900BB
:104100008091F000877F8093F00078940E94A62031
:104110001092E9008091F00088608093F000CD2B30
:10412000CF70C093E900FF91EF91DF91CF91BF91E4
:10413000AF919F918F917F916F915F914F913F913F
:104140002F910F900FBE0F901F9018951F93CF9334
:10415000DF93CDB7DEB7AA970FB6F894DEBF0FBED8
:10416000CDBFEBE9F2E08091F100819322E0E33AE8
:10417000F207C9F70E94AD1B8091E80083FF2EC1B2
:1041800080919B0290919C02492F50E04A3051054A
:1041900008F024C1FA01EE59FF4F0C942D2280380B
:1041A00021F0823809F01AC108C0809197029091DD
:1041B0009802992389F082600FC080919F028F70CE
:1041C000873008F00BC18093E9008091EB0085FBFC
:1041D000882780F91092E9009091E800977F9093EA
:1041E000E8008093F1001092F100D1C0282F2D7FBC
:1041F00009F0F4C0882319F0823061F0EFC080919B
:104200009D02813009F0EAC0933009F080E080938C
:1042100098022EC080919D0281112AC080919F0238
:104220008F702FEF280F263008F0D8C08093E90058
:104230002091EB0020FF1CC0933021F48091EB0013
:10424000806214C09091EB0090619093EB0021E0AC
:1042500030E0A90102C0440F551F8A95E2F7409350
:10426000EA001092EA008091EB0088608093EB00F6
:104270001092E9008091E800877F8093E8000E9417
:10428000C31EACC08111AAC010919D021F778091FE
:10429000E3008078812B8093E3008091E800877FA2
:1042A0008093E8000E94C31E8091E80080FFFCCF4D
:1042B0008091E30080688093E300111102C082E0E6
:1042C00001C083E080939A0289C08058823008F050
:1042D00085C080919D0290919E028C3D53E0950790
:1042E00079F583E08A838AE289834FB7F894DE0107
:1042F000139620E03EE051E2E32FF0E050935700A8
:10430000E49120FF03C0E295EF703F5FEF708E2FC6
:1043100090E0EA3010F0C79601C0C0968D939D934F
:104320002F5F243149F74FBF8091E800877F80934A
:10433000E8006AE270E0CE0101960E94CF1D16C02F
:1043400060919F027091A002AE014F5F5F4F0E948B
:10435000161DBC01892B09F441C09091E800977F9C
:104360009093E80089819A810E942D1E8091E80037
:104370008B778093E80032C0803881F58091E80027
:10438000877F8093E800809196028093F10080916E
:10439000E8008E7772CF811121C080919D029091AB
:1043A0009E0299270297D4F48091E800877F80933A
:1043B000E80080919D02809396020E94C31E809126
:1043C0009602811106C08091E30087FD02C081E062
:1043D00001C084E080939A020E94941B8091E800BF
:1043E00083FF0AC08091E800877F8093E800809176
:1043F000EB0080628093EB00AA960FB6F894DEBFC4
:104400000FBECDBFDF91CF911F910895CF938091C3
:104410009A028823A1F0C091E900CF709091EC003E
:10442000892F817090FD80E8C82B1092E90080915F
:10443000E80083FD0E94A620CF70C093E900CF91D1
:104440000895991B79E004C0991F961708F0961BF0
:10445000881F7A95C9F780950895EE0FFF1F059084
:10446000F491E02D0994FB01DC0104C08D910190D1
:10447000801921F441505040C8F7881B990B0895CA
:10448000F999FECF92BD81BDF89A992780B508951C
:10449000A8E1B0E042E050E00C947422262FF99994
:1044A000FECF92BD81BDF89A019700B4021639F093
:1044B0001FBA20BD0FB6F894FA9AF99A0FBE089564
:1044C0000396272F0E944F220E944E22252F0E94E2
:1044D0004F22242F0C944F220196272F0E944F2207
:1044E0000C944E22DC01CB01FC01F999FECF06C0F1
:1044F000F2BDE1BDF89A319600B40D9241505040A2
:08450000B8F70895F894FFCF0D
:10450800C8001602A11AA51A191B151B111BA41AFB
:1045180001E200E900EA00B500B600B700CD00836B
:1045280001CC008A01920194012102230224022570
:1045380002260227022A02B300B4006F007000812D
:104548008283E200E900EA00B500B600B700CD00BA
:104558008301CC008A0192019401210223022402E2
:104568002502260227022A02B300B4006F00700059
:10457800818283F1F03067F4F5F6F79496349790DA
:10458800953536406D22AB053E051C05C104DA049D
:02459800F3042A
:00000001FF
